:40000000021FC9008F828E83E0540100000070F82278FFE4F6D8FD022027EC4D6011E8497017ED33EC3304600DE4FCFFFEFD22E933E8330470F80202E31202AE5804600967
:40004000E4CC248150062850090202ED2840030202EAC0E0EB4A7044B98006D0E0FB0202D9EF4E701CBD8008EBFFEAFEE9FD80EBE98DF0A4FEE5F0020103E9CDF9EAFEEB24
:40008000FFEF89F0A4FCE5F0CE89F0A42EFFE435F0CD89F0A42DFEE435F08067EF4E7005BD80D780C3EF8BF0A4ACF0EE8BF0A42CFCE435F0F8EF8AF0A42CE5F038FCE433FC
:4000C000CB8DF0A42CFCE5F03BF8EE8AF0A42CFCE5F038F8E433CF89F0A42CFCE5F038CF3400CE89F0A42FFFE5F03EFEE433C98DF0A42EFEE5F039CD8AF0A42FFFE5F03EDF
:40010000FEE43DFD33D0E0FB50070BBB000F0202EDEC2CFCEF33FFEE33FEED33FD0202C50202EDEC5D046005E8590470030202E31202AE580460F6EC4860F2EC7004FDFED7
:40014000FF22C860DB2481C85009C398600250060202EA9850CAF582E9294B4A7005AB820202D975F0007C1A7880C3EF9BEE9AED99400DC3EF9BFFEE9AFEED99FDE842F03B
:40018000DC23ACF0D0E0FFD0E0FED0E0FDAB8220E7101BEB60BAEC2CFCEF33FFEE33FEED33FD0202C5E803F830E705C0F075F000EF2FFFEE33FEED33FD40B830E7C280AA94
:4001C00074F8CC6480CCC86480C8F58204604FC3EB9FF5F0EA9E42F0E99D42F0E89C45F0603C501DE5825FFFE582D313CB5BCBF42B5582FB50280ABA002409B90020088055
:400200001DE5825BFBE582D313CF5FCFF4C3132F5582FF50090EBE00050DBD00010CC3EB9FF5F0EA9E42F0E99D42F0E89C45F06007CC4820E701B3EC2275F020800E75F0B1
:4002400010800575F0087D007E007F003392D530D503120554EC334010EF33FFEE33FEED33FDEC33FCD5F0ED22E5F0247EA2D513CC92E7CDCEFF22EDD2E7CD33EC3392D50C
:4002800024814006E4FFFEFDFC22FCE4CFCECDCC24E0501174FF80EDC3CC13CCCD13CDCE13CECF13CF0470F030D5DE020554E9D2E7C933E833F892D5EDD2E7CD33EC33FC06
:4002C0005002B2D522EC30E7100FBF000C0EBE00080DBD00040BEB6014A2D5EB13FCED92E7FD2274FFFCFDFEFF22E480F8A2D574FF13FC7D80E480EFBB010689828A83E02A
:40030000225002E722BBFE02E32289828A83E49322BB010689828A83F0225002F722BBFE01F322EF8DF0A4A8F0CF8CF0A428CE8DF0A42EFE22BC000BBE0029EF8DF084FF10
:40034000ADF022E4CCF875F008EF2FFFEE33FEEC33FCEE9DEC984005FCEE9DFE0FD5F0E9E4CEFD22EDF8F5F0EE8420D21CFEADF075F008EF2FFFED33FD4007985006D5F065
:40038000F222C398FD0FD5F0EA22C2D5EC30E709B2D5E4C39DFDE49CFCEE30E715B2D5E4C39FFFE49EFE120335C3E49DFDE49CFC800312033530D507C3E49FFFE49EFE22DD
:4003C000C5F0F8A3E028F0C5F0F8E582158270021583E038F022BB010A89828A83F0E5F0A3F0225006F709A7F01922BBFE06F3E5F009F31922EF2BFFEE3AFEED39FDEC3812
:40040000FC22C3EF9BFFEE9AFEED99FDEC98FC22E88FF0A4CC8BF0A42CFCE98EF0A42CFC8AF0EDA42CFCEA8EF0A4CDA8F08BF0A42DCC3825F0FDE98FF0A42CCD35F0FCEB3F
:400440008EF0A4FEA9F0EB8FF0A4CFC5F02ECD39FEE43CFCEAA42DCE35F0FDE43CFC2275F008758200EF2FFFEE33FECD33CDCC33CCC58233C5829BED9AEC99E58298400C0F
:40048000F582EE9BFEED9AFDEC99FC0FD5F0D6E4CEFBE4CDFAE4CCF9A88222B800C1B90059BA002DEC8BF084CFCECDFCE5F0CBF97818EF2FFFEE33FEED33FDEC33FCEB33C4
:4004C000FB10D703994004EB99FB0FD8E5E4F9FA227818EF2FFFEE33FEED33FDEC33FCC933C910D7059BE99A4007EC9BFCE99AF90FD8E0E4C9FAE4CCFB2275F010EF2FFF10
:40050000EE33FEED33FDCC33CCC833C810D7079BEC9AE899400AED9BFDEC9AFCE899F80FD5F0DAE4CDFBE4CCFAE4C8F922EF5BFFEE5AFEED59FDEC58FC22EF4BFFEE4AFE29
:40054000ED49FDEC48FC22CFF4CFCEF4CECDF4CDCCF4CC22C3E49FFFE49EFEE49DFDE49CFC22EB9FF5F0EA9E42F0E99D42F0EC6480C864809845F022EB9FF5F0EA9E42F042
:40058000E99D42F0E89C45F022E8600FECC313FCED13FDEE13FEEF13FFD8F122E8600FEFC333FFEE33FEED33FDEC33FCD8F122E0FCA3E0FDA3E0FEA3E0FF22E0F8A3E0F959
:4005C000A3E0FAA3E0FB227401FF3395E0FEFDFCA3A3A3E02FFFF0E582158270021583E03EFEF0E582158270021583E03DFDF0E582158270021583E03CFCF022ECF0A3ED20
:40060000F0A3EEF0A3EFF022A42582F582E5F03583F58322E0FBA3E0FAA3E0F922EBF0A3EAF0A3E9F022E493FB740193FA740293F922D083D082F8E4937012740193700D1D
:40064000A3A393F8740193F5828883E4737402936860EFA3A3A380DFD083D082F8E4937012740193700DA3A393F8740193F5828883E473740293B5F0067403936860E9A3E1
:40068000A3A3A380D8E5162582F582E5153583F583B515048582162210AF06858216F51522858216F515D2AF22EC8EF0A4CCC5F0CCCDF8EFA4CEC5F02DFDE43CFCE8A42E9B
:4006C000C8C5F03DFDE43CFCEFA4FFE5F028FEE43DFDE43CFC22E709F608DFFA8046E709F208DFFA803E88828C83E709F0A3DFFA8032E309F608DFFA806EE309F208DFFA99
:40070000806688828C83E309F0A3DFFA805A89828A83E0A3F608DFFA804E89828A83E0A3F208DFFA804280D280FA80C680D4805580F28029801080A680EA809A80A880DA06
:4007400080E280CA802988848C8589828A83E493A30586F0A30586DFF5DEF3800B89828A83E493A3F608DFF9ECFAA9F0EDFB2288848C8589828A83E0A30586F0A30586DF2B
:40078000F6DEF480E389828A83E493A3F208DFF980D688F0EF60010E4E60CD88F0ED2402B4040050C3F582EB2402B4040050B92323458223900726734103390042012B0079
:4007C0000044011200000000420558000042055E000042056000004205550000608003D4000000000000000000000000000000000000000000000000000000000000000064
:4008000000000000000000000000000000000000000000000000000000000000000000000000000000000000000000000000000000000000000000000000000000000000B8
:400840000000000000000000000000000000000000000000000000000000000000000000608004540000000000000000000000000000000000000000000000000000000040
:400880000000000000000000000000000000000000000000000000000000000000000000000000000000000000000000000000000000000000000000000000000000000038
:4008C000000000000000000000000000000000000000000000000000000000000000000000000000608004D400000000000000000000000000000000000000000000000040
:4009000000000000000000000000000000000000000000000000000000000000000000000000000000000000000000000000000000000000000000000000000000000000B7
:400940000000000000000000000000000000000000000000000000000000000000000000000000000000000060800352000000000000000000000000000000000000000042
:400980000000000000000000000000000000000000000000000000000000000000000000000000000000000000000000000000000000000000000000000000000000000037
:4009C000000000000000000000000000000000000000000000000000000000000000000000000000000000000000000044011C0000000044012000000000440125000000C7
:400A00000044055A0000000041033600410131014101091F410566004203D20000410557004105540044033A0000000044033E0000000044034200000000440101000000EC
:400A4000004401050000000044010A0000000044010E00000000440562000000004405670000000044056B000000004403320000000044012D0000000042011600004201F4
:400A800018000042011A00004203500000410337014100001042012900004505FB050607080945060000010203044505F50506070809410634804106337F44062F00000463
:400AC000004106100041060B004106060041060C004106050141062D004105B4004105B5004105B300410642004106450041064600410647FF410648004106490044061A4C
:400B0000016E360044061500005DC04106191844061F2EE0000046063500010800180041064AFF43063B00000041064B0000C0E0C083C082C085C084C086758600C09375A6
:400B40009300C0D075D000C000C001C002C003C004C005C006C0079049D7E0FF900644EFF0900644E0FFEF5408FF7E00EF64084E70047F0180027F00EF7003020C0790493A
:400B8000D8E0FFEF5401FF7E00EF64014E70047F0180027F00EF604790062712061490062AE0FFE92FF9E43AFA1202F8FF9049D8EFF09049D77414F090062AE0FF90062EB9
:400BC000EFF090062EE004F0900624E0FFEF4411FF900624EFF09006237408F0020D659049D77410F0900624E0FFEF4412FF900624EFF09006237401F09049D6E0FFEF44F7
:400C000010FFEFF0020D65900644E0FFEF5401FF7E00EF64014E70047F0180027F00EF7003020D65900623E0FFEF1206320C3A010C85040CD60800000D519049D8E0FF9056
:400C40000643EFF0900643E0FF7E0090062BE0FCA3E0FDC3EF9DEE9C50239049D77410F0900643E0FF90062AEFF0900643E0FF90062EEFF09006237404F0020D659049D792
:400C8000E4F0020D6590062EE0FF7E00900625E0FCA3E0FDC3EF9DEE9C50339049D8E0FF900643EFF09049D77410F0900643E0FF90062712061490062EE0FEE92EF9E43A7B
:400CC000FAEF12031190062EE004F0020D659049D7E4F0020D65900644E0FFEF5402FF7E00EF4E704C90062EE0FF7E0090062BE0FCA3E0FDC3EF9DEE9C5028900627120609
:400D00001490062EE0FFE92FF9E43AFA1202F8FF9049D8EFF09049D77404F090062EE004F080429049D874FFF09049D77404F080349049D874FFF09049D7E4F0900624E0B4
:400D4000FFEF54EFFF900624EFF0900623E4F08014900623E4F090062AE4F090062EE4F09049D7E4F09049D7E0FFEF5420FF7E00EF64204E70047F0180027F00EF601E902A
:400D80000624E0FFEF54EFFF900624EFF0900623E4F09049D6E0FFEF54EFFFEFF0D007D006D005D004D003D002D001D000D0D0D093D086D084D085D082D083D0E0327B0095
:400DC0007A4679E81239ABEF4401FD7B007A4679E81239B7751400E514C3940A503AAF14EF75F005A42470F582E4343AF583AF82AE838E088F09AE08AF098F828E831206D3
:400E000026AE08AF098F828E83740393FC740493FD123713051480BF751400E514C394025078AF14EF75F008A424A2F582E4343AF583AF82AE838E0A8F0BAE0AAF0B8F82B6
:400E40008E831206268B0C8A0D890EAE0AAF0B8F828E83A3A3A31206268B0F8A108911AE0AAF0B8F828E83740693F512740793F513AB0FAA10A911C003C002C001AB0CAA42
:400E80000DA90E9005E012061DD001D002D003AF13AE121233A9051480817B087A0079001234CD905883740AF07B007A7679507D047C001237137B017A5079031239ABEF2E
:400EC0004402FD7B017A5079031239B77B017A5079131239ABEF4402FD7B017A5079131239B79043A0E0FFEF4440FF9043A0EFF09043C2E0FFEF4410FF9043C2EFF07B085A
:400F00007A097988C003C002C0017B007A5179009005E012061DD001D002D0037F0A7E001233A97B087A097994C003C002C0017B007A5179C09005E012061DD001D002D01E
:400F4000037F0A7E001233A97B087A0979A0C003C002C0017B007A5179229005E012061DD001D002D0037F087E001233A97B087A0979A8C003C002C0017B007A5179329032
:400F800005E012061DD001D002D0037F087E001233A97B087A0979B0C003C002C0017B007A5179429005E012061DD001D002D0037F087E001233A97B087A0979B8C003C06B
:400FC00002C0017B007A5179509005E012061DD001D002D0037F0A7E001233A99044F47401F0904322E0FFEF4408FF904322EFF09046ECE0FFEFC394055006904689743AAC
:40100000F090480074F1F012189C90480074B1F01231097B007A4379A0C003C002C0017B007A4379B09005E012061DD001D002D0037F0E7E001233A99043B0E0FFEF54FDE1
:40104000FFEFF0229005DDE4F0A3E4F07F007E007D007C0090011C1205FC7F007E007D007C009001201205FC7F007E007D007C009001251205FC7F007E007D007C009005F9
:401080005A1205FC9005DCE4F09005DCE0FFC3EF648094A040030211CA90011C1205AFC004C005C006C0079005DCE0FFEF3395E0FEEF7803C333CE33CED8F9FF74012FF53E
:4010C0008274003EF583E0FEA3E0FFAB07AA06E4F9F8D007D006D005D0041203F590011C1205FC9001201205AFC004C005C006C0079005DCE0FFEF3395E0FEEF7803C333BB
:40110000CE33CED8F9FF74032FF58274003EF583E0FEA3E0FFAB07AA06E4F9F8D007D006D005D0041203F59001201205FC9001251205AFC004C005C006C0079005DCE0FF2C
:40114000EF3395E0FEEF7803C333CE33CED8F9FF74052FF58274003EF583E0FEA3E0FFAB07AA06E4F9F8D007D006D005D0041203F59001251205FC90055A1205AFC004C099
:4011800005C006C0079005DCE0FFEF3395E0FEEF7803C333CE33CED8F9FF74072FF58274003EF583E0FEA3E0FFAB07AA06E4F9F8D007D006D005D0041203F590055A120571
:4011C000FC9005DCE004F0021089900109E004F0900109E0FFEF541FFF900109EFF0900566E004F0900566E0FFEF541FFF900566EFF090011C1205AF780512058990033615
:40120000E0FDED25E024D4F582E43403F583EEF0A3EFF09001201205AF7805120589900336E0FDED25E02454F582E43404F583EEF0A3EFF09001251205AF78051205899045
:401240000336E0FDED25E024D4F582E43404F583EEF0A3EFF090055A1205AF7805120589900336E0FDED25E02452F582E43403F583EEF0A3EFF0900336E004F0900336E073
:40128000FFEF543FFF900336EFF0900131E004F0900131E0FFEF543FFF900131EFF0229005E3EFF09005E4EDF09005E5EBF09005E7E4F09005E3E0FFEFC43354E0FF900534
:4012C000E4E0FEEF4EFF9005E7EFF0123A549005E3E0FFEF60030213689005E4E0FFEF640A60149005E4E0FFEF640B600A9005E4E0FFEF641070519005E7E0FF1233749066
:4013000005FAEFF09005E8E4F0A3E4F09005E8E0FEA3E0FFEF64054E60257FFF1233749005E8E0FCA3E0FD74F02DF58274053CF583EFF09005E8E475F0011203C080CD12E0
:401340003A4E9005FAE0FF229005E7E0FF1233749005FAEFF07FFF1233749005E6EFF0123A4E9005E6E0FF229005E3E0FFEF640160030214BC9005E4E0FFEF640A7059903E
:4013800005E7E0FF1233749005FAEFF09005EAE4F0A3E4F09005EAE0FEA3E0FFEF64054E602D9005EAE0FEA3E0FF74FB2FF58274053EF583E0FF9005E6EFF09005E6E0FFA9
:4013C0001233749005EAE475F0011203C080C5123A4E9005FAE0FF229005E4E0FFEF640B70599005E7E0FF1233749005FAEFF09005EAE4F0A3E4F09005EAE0FEA3E0FFEF8E
:4014000064054E602D9005EAE0FEA3E0FF74002FF58274063EF583E0FF9005E6EFF09005E6E0FF1233749005EAE475F0011203C080C5123A4E9005FAE0FF229005E4E0FF8E
:40144000EF641070599005E7E0FF1233749005FAEFF09005EAE4F0A3E4F09005EAE0FEA3E0FFEF64054E602D9005EAE0FEA3E0FF74F52FF58274053EF583E0FF9005E6EF7C
:40148000F09005E6E0FF1233749005EAE475F0011203C080C5123A4E9005FAE0FF229005E7E0FF1233749005E6EFF09005E5E0FF123374123A4E9005E6E0FF227F01229054
:4014C00005DCEFF09005DDECF0A3EDF09005DFEAF0A3EBF09005E2E0FFEFD3940050030216BE9005E2E0FFEFD3940140030216BE9005DCE0FFEF120632150C01150C041512
:401500003907156408158F0A000015BA9005E1E0FFEFD3940F40117B0C7A0179181239AB9005E3EFF00215BF7B0C7A01791C1239AB9005E3EFF00215BF9005E1E0FFEFD3DB
:40154000940F40107B0C7A0179191239AB9005E3EFF0806B7B0C7A01791D1239AB9005E3EFF0805B9005E1E0FFEFD3940F40107B0C7A01791A1239AB9005E3EFF080407BC5
:401580000C7A01791E1239AB9005E3EFF080309005E1E0FFEFD3940F40107B0C7A01791B1239AB9005E3EFF080157B0C7A01791F1239AB9005E3EFF080059005E3E4F09046
:4015C00005E3E0FFEF3395E0FEFDFC7B207A0079007800120410A804A905AA06AB079005DDE0FEA3E0FFE4FCFD1203F59005E41205FC9005E41205AFAB07AA06A905A8046E
:40160000A804A905AA06AB079005DFE0FEA3E0FFE4FCFD1204109005EA1205FC7B007A80790078009005EA1205AF12049B9005E8EEF0A3EFF09005E1E0FFEFC3940E50470C
:401640009005E8E0FEA3E0FF9005E1E0FDC3740E9DFDEFA805088005CEC313CE13D8F9FF9005E8EEF0A3EFF09005E1E0FFEF04FF9005E2E0FEEE75F003A4240CF582E434AB
:4016800006F583EFF080169005E2E0FFEF75F003A4240CF582E43406F583740FF09005E8E0FEA3E0FF9005E2E0FDED75F003A4240AF582E43406F583EEF0A3EFF0227F00D0
:4016C0001237F0229005DFE4F0A3E4F07F007E007D007C0090011C1205FC7F007E007D007C009001201205FC7F007E007D007C009001251205FC7F007E007D007C00900516
:401700005A1205FC9005DDE4F0A3E4F09005DDE0FEA3E0FFC3EF9420EE64809480400302184F90011C1205AFC004C005C006C0079005DDE0FEA3E0FFEF7803C333CE33CE2B
:40174000D8F9FF74012FF58274003EF583E0FEA3E0FFAB07AA06E4F9F8D007D006D005D0041203F590011C1205FC9001201205AFC004C005C006C0079005DDE0FEA3E0FF3E
:40178000EF7803C333CE33CED8F9FF74032FF58274003EF583E0FEA3E0FFAB07AA06E4F9F8D007D006D005D0041203F59001201205FC9001251205AFC004C005C006C00796
:4017C0009005DDE0FEA3E0FFEF7803C333CE33CED8F9FF74052FF58274003EF583E0FEA3E0FFAB07AA06E4F9F8D007D006D005D0041203F59001251205FC90055A1205AF5A
:40180000C004C005C006C0079005DDE0FEA3E0FFEF7803C333CE33CED8F9FF74072FF58274003EF583E0FEA3E0FFAB07AA06E4F9F8D007D006D005D0041203F590055A127E
:4018400005FC9005DDE475F0011203C002170C90011C1205AF7805120589900116EEF0A3EFF09001201205AF7805120589900118EEF0A3EFF09001251205AF7805120589E4
:4018800090011AEEF0A3EFF090055A1205AF7805120589900350EEF0A3EFF0227B007A4079807D007C0012392C9040827450F07B007A4079847D017C0012392C90408674D5
:4018C00018F07B007A4079887D0B7C0012392C90408A7418F07B007A40798C7D177C0012392C90408E7418F07B007A4079907D177C0012392C9040927418F07B007A40796D
:40190000947D197C0012392C9040967418F07B007A4079987D5F7CEA12392C90409A7419F07B087A0979C4C003C002C0017B007A4179009005E012061DD001D002D0037FEB
:40194000047E001233A99043007402F09040007408F09042007403F07B0C7A0179081239AB9046A1EFF07B007A4279227D087C0012392C7B007A4279207D517C1212392C8D
:401980009005DAE4F07F197E007D007C009005D61205FC9005D61205AFD3EF9400EE9400404E9005DAE0FFEF64036044904225E0FFEF5401FF7E009005DAE0FEEE25E0FEA3
:4019C000EE4FFFEF5403FF9005DAEFF07FE07E017D007C001234009005D61205AF7BFF7AFF79FF78FF1203F59005D61205FC80A39005D61205AFEF4E70057F0312382B7BE8
:401A0000007A4079047D007C0112392C9040047407F0904006E4F09040087448F0904004E4F09040017402F090400B7404F09043A2E0FFEF447FFF9043A2EFF09043A1E0C2
:401A4000FFEF4401FF9043A1EFF09043A0E0FFEF4480FF9043A0EFF0229005DDEEF0A3EFF09005DFEDF01239F79005E1EFF01239ED9005E2EEF0A3EFF09005E2E0FEA3E0C8
:401A8000FF9005DDE0FCA3E0FDED6F7002EC6E7003021BED9043A2E0FFEF5401FF9005E0EFF09005E1E0FFEF705E9005E2E0FEA3E0FFEF4E600C9005DDE0FEA3E0FFEF4E28
:401AC00070469005E2E0FEA3E0FFEF4E701D7B027A4079809005DDE0FCA3E0FD12392E904082E0FFEF54BFFFEFF022904082E0FFEF4440FFEFF07B027A4079809005DDE0E1
:401B0000FCA3E0FD12392E229005E0E0FFEF606C904001E4F09040107401F0904014E4F0904008E0FFEF547FFFEFF0904082E0FFEF5408FF7E00EF4E600C9005DDE0FEA3F1
:401B4000E0FFEF4E70367B027A4079029005E2E0FCA3E0FD12392E9040017407F0904001E0FFEF5401FF7E00EF4E70F19043A2E0FFEF54FEFFEFF0904001E4F09043A2E0ED
:401B8000FFEF5401FF7E00EF4E603A7B027A4079029005DDE0FCA3E0FD12392E9005DFE0FFEF60047F0280027F00EF4401FF904001EFF0904001E0FFEF5401FF7E00EF4EDC
:401BC000602B80EF227B027A4079809005DDE0FCA3E0FD12392E9043A2C083C082E0FF9005E0E0FEEF4EFFD082D083EFF0229005DDEEF0A3EFF09005DFEDF0123A0B900535
:401C0000E1EFF0123A019005E2EEF0A3EFF09005E2E0FEA3E0FF9005DDE0FCA3E0FDED6F7002EC6E7003021D829043A1E0FFEF5401FF9005E0EFF09005E1E0FFEF705E9053
:401C400005E2E0FEA3E0FFEF4E600C9005DDE0FEA3E0FFEF4E70469005E2E0FEA3E0FFEF4E701D7B027A4179009005DDE0FCA3E0FD12392E904102E0FFEF54BFFFEFF02262
:401C8000904102E0FFEF4440FFEFF07B027A4179009005DDE0FCA3E0FD12392E229005E0E0FFEF606C904001E4F09040147401F0904010E4F0904008E0FFEF547FFFEFF0FF
:401CC000904102E0FFEF5408FF7E00EF4E600C9005DDE0FEA3E0FFEF4E70367B027A4079029005E2E0FCA3E0FD12392E9040017407F0904001E0FFEF5401FF7E00EF4E70B4
:401D0000F19043A1E0FFEF54FEFFEFF0904001E4F09043A1E0FFEF5401FF7E00EF4E603A7B027A4079029005DDE0FCA3E0FD12392E9005DFE0FFEF60047F0280027F00EFA0
:401D40004401FF904001EFF0904001E0FFEF5401FF7E00EF4E602B80EF227B027A4179009005DDE0FCA3E0FD12392E9043A1C083C082E0FF9005E0E0FEEF4EFFD082D083A1
:401D8000EFF0229005DCE4F09005DDE4F0A3E4F09003D4E0FEA3E0FF9003F2E0FCA3E0FDC3ED9FFFEC9EFE9005DDEEF0A3EFF09005DDE0FEA3E0FF1239C3900000E0FD7C07
:401DC00000C3EF9DEC6480F8EE64809850069005DCE004F09003F2E0FEA3E0FF900412E0FCA3E0FDC3ED9FFFEC9EFE9005DDEEF0A3EFF09005DDE0FEA3E0FF1239C39000C8
:401E000000E0FD7C00C3EF9DEC6480F8EE64809850069005DCE004F0900412E0FEA3E0FF900432E0FCA3E0FDC3ED9FFFEC9EFE9005DDEEF0A3EFF09005DDE0FEA3E0FF1279
:401E400039C3900000E0FD7C00C3EF9DEC6480F8EE64809850069005DCE004F0900432E0FEA3E0FF900452E0FCA3E0FDC3ED9FFFEC9EFE9005DDEEF0A3EFF09005DDE0FE01
:401E8000A3E0FF1239C3900000E0FD7C00C3EF9DEC6480F8EE64809850069005DCE004F09005DCE0FFEFB404079003377401F022900337E4F0229005DCE4F07F001238DD93
:401EC0001237C69005DCE0FFEFC394404003021FC8900557E0FFEFB401E91216C4900557E4F0123A2C9005DCE004F09005DCE0FFEFB43FCF1239937F011238DD900109747C
:401F00001FF0900566E4F09005DCE004F090011C1205AFC004C005C006C007900116E0FEA3E0FFAB07AA06E4F9F8D007D006D005D00412040290011C1205FC9001201205C1
:401F4000AFC004C005C006C007900118E0FEA3E0FFAB07AA06E4F9F8D007D006D005D0041204029001201205FC9001251205AFC004C005C006C00790011AE0FEA3E0FFABE2
:401F800007AA06E4F9F8D007D006D005D0041204029001251205FC90055A1205AFC004C005C006C007900350E0FEA3E0FFAB07AA06E4F9F8D007D006D005D004120402901B
:401FC000055A1205FC021EC32275930078007583467582E8E04401F0009046ECE0F99046FAE0FAB903225420B40012B8001AEA901FFFF07401901FFEF09046F6F0901FFE86
:40200000E06005901FFFE0FA90480074C0F075811690000078007920E4F0A3D8FCD9FAEA90061EF002001175151F7516FD120DBE12315702207102233AE493A3F8E493A3A5
:402040004003F68001F208DFF48029E493A3F85407240CC8C333C4540F4420C8834004F456800146F6DFE4800B01020408102040809007B8E47E019360BCA3FF543F30E5BC
:4020800009541FFEE493A360010ECF54C025E060A840B8E493A3FAE493A3F8E493A3C8C582C8CAC583CAF0A3C8C582C8CAC583CADFE9DEE780BE9005DCEFF090060BE4F06C
:4020C0009005DCE0FFEF64016003022199904E007432F0904E027406F0904E037408F0904E04E4F0904E05E4F0904E06741FF0904E08E4F0904E09E4F0904E0AE4F0904E2F
:40210000147401F09058847414F09058857406F09058867414F0905887E4F090588A7444F090588B7448F090588C7401F090588E7402F090588F7422F09058907428F090C3
:40214000589174EBF07F531230659058947458F0905895E4F090589A7405F090589B7402F090589CE4F090589DE4F07F0012360F7FD97E047D007C009006111205FC7D01BF
:402180007F097E00121A597D017F277E00121BEE7C3A7D667F1D122C28229005DC12061D9005DFECF0A3EDF09005DC1206149005DFE0FCA3E0FD122BA012393B123A5A7DB1
:4021C000FF7FFF1229309005E1EFF09005E1E0FFEF20E53A9005E1E0FFEF30E4239005E1E0FFEF4410FB7D077F0112129F9005E2EFF07DFF7FFF1229309005E1EFF0800EAC
:402200007DFF7FFF1229309005E1EFF080BD9005E1E0FFEF30E5159005E1E0FFEF4420FB7D077F0112129F9005E2EFF09005E1E0FFEF30E4159005E1E0FFEF4410FB7D07F5
:402240007F0112129F9005E2EFF09005E1E0FFEF30E00C7DFF7FE11229309005E2EFF07DFF7FFF1229309005E1EFF0221237879005DDEFF0900605E0FF9005DCEFF090432E
:40228000AAE0FFEF4401FFEFF09043AAE0FFEF4410FFEFF09043BAE0FFEF4401FFEFF09043BAE0FFEF4410FFEFF09046F8E0FFEF4402FFEFF09046F9E0FFEF4402FFEFF07A
:4022C000905891E0FFEF4403FFEFF07F037E001234A09046F8E0FFEF54FDFFEFF09046F9E0FFEF54FDFFEFF0905877E0FFEF4406FFEFF0905882747AF09043A1E0FFEF44D2
:4023000001FFEFF09043B1E0FFEF4401FFEFF09043A2E0FFEF4401FFEFF09043B2E0FFEF4401FFEFF09044DB7420F09044C37420F09005DDE0FF12372C227BFF7A3A794848
:402340009005D712061D9005DAE4F09005DBE4F01233DD123A5A7DFF7FE11229309005D6EFF0121EB6123A1512396F900557E0FFEFB4012312259E121044900557E4F0123C
:402380003A2C121D83122EE11234FA900337E0FFEFB401031216C4900554E0FFEFB401CB900554E4F0123A419005621205AF120554AB07AA069001051205AFEB2FFFEA3EC0
:4023C000FE12265E900113EFF01236E0EF700A122407900115EFF08005900115E4F09001051205AF9005621205FC9003321205AF90012D1205FC7B017A0179127D047C0033
:4024000012219A02236B229005DCE4F0A3E4F0900336E0FFEF7021900350E0FEA3E0FF9003D0E0FCA3E0FDC3ED9FFFEC9EFE9005DCEEF0A3EFF0802D900336E0FFEF25E047
:402440002450F582E43403F583E0FEA3E0FF900350E0FCA3E0FDC3EF9DFFEE9CFE9005DCEEF0A3EFF09005DCE0FEA3E0FF1239C3C3EF94F4EE6480948150199005DCE0FEE0
:40248000A3E0FF7C007D2812038A9005DCEEF0A3EFF080379005DCE0FEA3E0FF1239C3C3EF94E8EE6480948350199005DCE0FEA3E0FF7C007D1912038A9005DCEEF0A3EF90
:4024C000F080089005DCE4F0A3E4F09005DCE0FEA3E0FF229006057401F0900610E4F07F101235747F101235957D077F1D122FAC9058967407F0905897E4F090589EE4F0E3
:40250000905B07E0FFEF4418FFEFF0905893E4F0905B88E4F0905B89E4F0905880740AF0905881E4F0905883E4F09058887412F09058897413F090588DE4F0904E017414F3
:40254000F09005E1740CF09005E27401F07B007A807D007C907F021214BF900605E0FFEF75F003A4240CF582E43406F583E0FF904E0EEFF0900605E0FFEF75F003A4240A46
:40258000F582E43406F583E0FCA3E0FD7B027A4E790C12392E900605E0FF1220B6229005DCE4F0A37401F09005DCE0FEA3E0FFC3EF943FEE64809480400302265D9005DC29
:4025C000E0FEA3E0FFEF25E0FFEE33FE74502FF58274033EF583E0FCA3E0FD9005DCE0FEA3E0FFEF25E0FFEE33FE74522FF58274033EF583E0FEA3E0FFC3EF9DFBEE9CFACC
:402600009005DCE0FEA3E0FFEF25E0FFEE33FE74502FF58274033EF583E0FEA3E0FF7C007D091203237C007D0A120335EF2BFDEE3AFC9005DCE0FEA3E0FFEF25E0FFEE3319
:40264000FE74522FF58274033EF583ECF0A3EDF09005DCE475F0011203C00225A7229005DCEEF0A3EFF09005DCE0FEA3E0FF1239C3C3EF9432EE6480948050109005DCE028
:40268000FEA3E0FF7C007D0C12038A229005DCE0FEA3E0FF1239C3C3EF9420EE6480948350109005DCE0FEA3E0FF7C007DA012038A229005DCE0FEA3E0FF1239C3C3EF94F6
:4026C00040EE6480949F50109005DCE0FEA3E0FF7C037D2012038A229005DCE0FEA3E0FF1239C3EE3395E0FDFC7B807A3879017800D312056240109005DCE0FEA3E0FF7C91
:40270000137D8812038A229005DCE0FEA3E0FF1239C37C307DD412038A22123A5A7B0A7D007F0112129F9005FAEFF07B037D037F0112129F9005FAEFF07BF37D047F01129A
:40274000129F9005FAEFF07BFF7D107F0112129F9005FAEFF07BFF7D0A7F0112129F9005FAEFF07BFF7D0A7F0012129F9005FAEFF07B017D017F0112129F9005FAEFF07BF9
:40278000017D027F0112129F9005FAEFF07B047D117F0112129F9005FAEFF07B017D0B7F0112129F9005FAEFF07B017D1D7F0112129F9005FAEFF07B0E7D067F0112129F5F
:4027C0009005FAEFF07B327D057F0112129F9005FAEFF0229005E2EFF09005E3EDF09005E4EBF09005E87401F09005E2E0FFEFC3941840030228879005E4E0FFEF5401FF45
:402800007E00EF75F080A4FFAEF09005E3E0FEEE547FFEEE4FFF9005E2E0FE75F008EE907600120608EFF09005E6E0FFEF540FFF7E00EF75F010A4FFAEF09005E5E0FEEEEB
:40284000540FFEEE4FFF9005E2E0FE75F008EE907601120608EFF09005E7E0FFEF540FFF9005E2E0FE75F008EE907602120608EFF09005E2E0FF75F008EF907603120608C7
:40288000E4F09005E8E4F09005E8E0FF229005DCEFF09005DDECF0A3EDF09005DFEBF09005E17401F09005DCE0FFEFC39480507A9005DDE0FEA3E0FFEE54F0FE7F00EF4E8F
:4028C00070689005DCE0FF7E08EF8EF0A4FFAEF0EF2400FFEE3478FE9005E2EEF0A3EFF09005E2E0FEA3E0FFAA06A9077B019005DDE0FCA3E0FD12392E9005DFE0FF900519
:40290000DCE0FE75F008EE907802120608EFF09005E0E0FF9005DCE0FE75F008EE907803120608EFF09005E1E4F09005E1E0FF229005E3EFF09005E4EDF09005E5E4F012A3
:402940003A549005E3E0FFEFB461209005E3E0FF1233749005FAEFF07FFF1233749005E5EFF0123A4E9005E5E0FF229005E3E0FFEFB4A01E9005E3E0FF1233749005FAEFE5
:40298000F09005E4E0FF123374123A4E9005FAE0FF229005E3E0FFEFB4B01E9005E3E0FF1233749005FAEFF09005E4E0FF123374123A4E9005FAE0FF229005E3E0FF1233CF
:4029C000749005FAEFF0123A4E9005FAE0FF229005E2EFF09005E3ECF0A3EDF09005E5EAF0A3EBF09005E77401F09005E2E0FFEFC3941850739005E2E0FF7E08EF8EF0A48A
:402A0000FFAEF0EF2404FFEE3476FE9005E8EEF0A3EFF09005E8E0FEA3E0FFAA06A9077B019005E3E0FCA3E0FD12392E9005E2E0FF7E08EF8EF0A4FFAEF0EF2406FFEE34A6
:402A400076FE9005E8EEF0A3EFF09005E8E0FEA3E0FFAA06A9077B019005E5E0FCA3E0FD12392E9005E7E4F09005E7E0FF229005DCEFF09005DDECF0A3EDF09005DFEAF0C4
:402A8000A3EBF09005E17401F09005DCE0FFEFC3948050739005DCE0FF7E08EF8EF0A4FFAEF0EF2404FFEE3478FE9005E2EEF0A3EFF09005E2E0FEA3E0FFAA06A9077B0128
:402AC0009005DDE0FCA3E0FD12392E9005DCE0FF7E08EF8EF0A4FFAEF0EF2406FFEE3478FE9005E2EEF0A3EFF09005E2E0FEA3E0FFAA06A9077B019005DFE0FCA3E0FD12EF
:402B0000392E9005E1E4F09005E1E0FF22C0E0C083C082C085C084C086758600C093759300C0D075D000C006C007A2AFE433FF9005EFEFF0D2AF9044F474FDF09005B3E025
:402B4000FF9005B5E0FEEE6F6037906566E0FFEF20E22E9005B5E0FFEFC3942040059005B5E4F09005B5E0FF74B62FF582E43405F583E0FF906545EFF09005B5E004F080CB
:402B8000BB9005EFE0FFEF24FF92AFD007D006D0D0D093D086D084D085D082D083D0E0329005E312061D9005E6ECF0A3EDF0123A547FA01233749005E9E4F0A3E4F0900514
:402BC000E6E0FEA3E0FF9005E9E0FCA3E0FDC3ED9FEE6480F8EC64809850449005E31206149005E9E0FEA3E0FFE92FF9EA3EFA1202F8FF1233749005E31206149005E9E025
:402C0000FEA3E0FFE92FF9EA3EFA1202F8FF9005E8EFF09005E9E475F0011203C0809F123A4EE47E007F00229005DDEFF09005DEECF0A3EDF09005DDE0FFEFD3941F5003E8
:402C4000D38001C340057F001237F09005DDE0FFEF541FFF7E00EF25E0FFEE33FEEF2400FFEE3444FEAA06A9077B0112391F9005E0EEF0A3EFF09005DDE0FF7E02EF8EF02F
:402C8000A4FFAEF0EF2400FFEE3444FEAA06A9077B019005DEE0FEA3E0FFAD07AC0612392E9005E0E0FEA3E0FF229005E0E4F0A3E4F07B007A007D017F02122F4B900124E3
:402CC000EFF01231A4900338EFF0900338E0FF900338E0FB9005E07482F07D007C0112288D900338E0FFC0077B017A007901AF01AE02AD037C00EF54FFFFEE54FFFEED54CA
:402D000000FDEC5400FCAB07AA06D0077D107C4E122A6E900124E0FF900338E0FD1232C6900124E0FF7D01122D2B229005DCEFF09005DDEDF09005DE7401F09005DCE0FF75
:402D4000EFC3941850549005DDE0FFEF60199005DCE0FF75F010EF907010120608E0FFEF4420FFEFF080179005DCE0FF75F010EF907010120608E0FFEF54DFFFEFF09005B5
:402D8000DCE0FF75F010EF907010120608E0FFEF4401FFEFF09005DEE4F09005DEE0FF229005E2EFF09005E3EDF09005E57401F09005E2E0FFEFC39418504A9005E2E0FFEA
:402DC00075F010EF907010120608E0FFEF54F1FF9005E4EFF09005E3E0FFEF5407FF7E00EF25E0FFEE33FE9005E4E0FEEF4EFF9005E2E0FE75F010EE907010120608EFF04B
:402E00009005E5E4F09005E5E0FF22906575E0FFEF54C0FF9005DDEFF09005DDE0FFEF4409FF906575EFF0906496E0FFEF4401FFEFF0906497E0FFEF4401FFEFF07FF97E6B
:402E4000001236447FF97E0012365E7F7D7E001236787F001238BD1237879005DEEFF0906496E0FFEF4410FFEFF09005DEE0FF12372C12395522906477E0FFEF54C0FF9059
:402E800005DCEFF09005DCE0FFEF4409FF906477EFF0906596E0FFEF4401FFEFF0906597E0FFEF4401FFEFF07F0F7E271236927F0F7E271236AC7F887E131236C67F001219
:402EC00038ED1237879005DDEFF0906497E0FFEF4410FFEFF09005DDE0FF12372C12396222900337E0FFEF705390033A1205BB900116E0FEA3E0FF900412E0FCA3E0FDC3A6
:402F0000ED9FFFEC9EFEE4FCFD1203F590033A1205FC9003321205BB900116E0FEA3E0FF900390E0FCA3E0FDC3ED9FFFEC9EFEE4FCFD1203F59003321205FC227F007E00E6
:402F40007D007C0090033A1205FC229005DCEFF09005DDEDF09005DEEAF0A3EBF0900647740AF0900647E0FF9005DCE0FD9005DDE0FB9005E5E4F09005E6E4F09005E7E44D
:402F8000F01227D4900647E0FF9005DEE0FCA3E0FD9005E0E0FAA3E0FB1229CF900647E0FF7D02122DA0900647E0FF229005DCEFF09005DDEDF09005DDE0FFEFD39407501D
:402FC00003D38001C340057F001237F09005DCE0FFEFD3941F5003D38001C340057F001237F09005DDE0FFEF5407FF7E00EF75F020A4FFAEF09005DCE0FEEE541FFE74801F
:403000002EF582E43444F583EFF02290647BE0FFEF54C0FF9005DCEFF09005DCE0FFEF4409FF90647BEFF0906498E0FFEF4401FFEFF07F3212386D7F3212387D7F1912385E
:403040008D7F0012389D1237879005DDEFF0906498E0FFEF4410FFEFF09005DDE0FF12372C123948229005DDEFF01237879005DEEFF09046F8E0FFEF4403FFEFF09046F932
:40308000E0FFEF4403FFEFF09005DDE0FF905892EFF07F037E001234A09046F8E0FFEF54FCFFEFF09046F9E0FFEF54FCFFEFF09005DEE0FF12372C22C0E0C083C082C085A5
:4030C000C084C086758600C093759300C0D075D000C007900648E0FFEF5403FF900648EFF0900648E0FFEFB403069005577401F0900648E004F0D007D0D0D093D086D084A5
:40310000D085D082D083D0E0327B0C7A0179CF1239AB9005D6EFF09005D6E0FFEF5407FF90586EEFF09005D6E0FFEFC4540FFFEF540FFF90586FEFF090510D7402F0905146
:403140003D74E0F0905B0074E0F0905B5874E0F09058767466F022900633747FF09006347480F09005D6747FF09005D6E0FFEF60219005D6E0FFEF14FF9005D6E0FE75F072
:4031800008EE907800120608EFF09005D6E014F080D79005D6E0FF75F008EF907800120608E4F0229005DD74FFF01237879005DCEFF0900634E0FFEFD3941840269006336D
:4031C000E0FF9005DDEFF0900634E014F09005DDE0FF75F008EF907800120608E0FF900633EFF09005DCE0FF12372C9005DDE0FF229005DFEFF09005DFE0FFEFC39402501F
:40320000399005DFE0FFEF25E0246AF582E4343AF583E493FE740193FF8F828E83C083C082E0FF9005DFE0FEEE903A6E93FEEEF4FEEF5EFFD082D083EFF0229005DEEFF010
:403240009005DEE0FFEFC3940250369005DEE0FFEF25E0246AF582E4343AF583E493FE740193FF8F828E83C083C082E0FF9005DEE0FEEE903A6E93FEEF4EFFD082D083EF3F
:40328000F022C2D5E830E70FB2D5E4C39BFBE49AFAE499F9E498F8EC30E717B2D51232B812049BE4C39BFBE49AFAE499F9E498F8800312049B30D50DE4C39FFFE49EFEE455
:4032C0009DFDE49CFC229005DCEFF09005DDEDF09005DE7401F09005DCE0FFEFC39418501B9005DDE0FF9005DCE0FE75F010EE907019120608EFF09005DEE4F09005DEE051
:40330000FF221237879005DCEFF090649AE0FFEF4420FFEFF0906599E0FFEF4410FFEFF0906499E0FFEF4410FFEFF09005DCE0FF12372C12374412349E12349F22906469F9
:40334000E0FFEF30E50790645AE0FF80F01237879005DCEFF090649AE0FFEF4401FFEFF090649AE0FFEF54FEFFEFF09005DCE0FF12372C229005ECEFF09005EDE4F0900569
:40338000ECE0FF1236FA906469E0FF9005EDEFF09005EDE0FFEF20E50C906469E0FF9005EDEFF080EB12385D22758600EF4E6027EF60010E7593009005E0E0F595A3E0F5B5
:4033C00085A3E0F5848B938A838982E0A30586F0A31586DFF6DEF4E4F593F59522D2AF9044F474FDF01237B11239CF7FF37E0112365E7FFA7E0012367812379C12271A22B5
:40340000EC4D4E700D78FCEF24E950032840FD2200007BF178DA0000EF28FF78FFEE38FEED38FDEC38FC50E7EF2BFFEE38FEED38FDEC38FC40F222050203049005ECEFF015
:403440009051C0E0FFEF547FFF9005EDEFF09005ECE0FFEFC43333335480FFEF5480FF9005EDE0FEEF4EFF9051C0EFF0229005E3EFF09051C0E0FFEF54BFFF9005E4EFF0FB
:403480009005E3E0FFEFC4333354C0FFEF5440FF9005E4E0FEEF4EFF9051C0EFF0222222EEFA900619E0F88FF0A4FFAEF0E88AF0A42EFEE5F03400FDEF24C9FF78FFEE38AF
:4034C000FEED38FDE438FC500302340022ACEAADA08B938A838982E0F96017A3E0F5EAA3E0F5A0A3E060F4FAA3E0F8A3E0F2DAF8D9E98DA08CEAE4F593229001051205AF24
:403500009005621205FC900337E0FFEF70159001051205AF90033A1205BB1203F59001051205FC22C0E0C083C082C085C084C086758600C0937593009005547401F0D09399
:40354000D086D084D085D082D083D0E0329005DEE4F09005DEE0FFEFC3940250109005DEE0FF1231F19005DEE004F080E590064A74FFF0229005DCEFF0904082C083C082C6
:40358000E0FF9005DCE0FEEE54F8FEEF4EFFD082D083EFF0229005DCEFF0904102C083C082E0FF9005DCE0FEEE54F8FEEF4EFFD082D083EFF0229005DCEEF0A3EFF07B0285
:4035C0007A4479049005DCE0FEA3E0FFAD07AC0612392E229005DCEEF0A3EFF07B027A4479029005DCE0FEA3E0FFAD07AC0612392E22900606E0FFEF701190060CE0FFEF0A
:4036000070031224D49006067401F012226C229005DDEFF012354D9005DDE0FF12323B9005DDE0FF90064AEFF02290648A740FF012333D12383D12384D906589E4F090648C
:4036400089E4F0229005DFEEF0A3EFF07B027A6479069005DFE0FCA3E0FD12392E229005DFEEF0A3EFF07B027A6479469005DFE0FCA3E0FD12392E229005DFEEF0A3EFF085
:403680007B027A6479269005DFE0FCA3E0FD12392E229005DEEEF0A3EFF07B027A6579069005DEE0FCA3E0FD12392E229005DEEEF0A3EFF07B027A6579469005DEE0FCA3AD
:4036C000E0FD12392E229005DEEEF0A3EFF07B027A6579269005DEE0FCA3E0FD12392E22905101E0FFEF5410FF7E00EEC4F854F0C868FEEFC4540F48FF229005EEEFF090FC
:403700006569E0FFEF30E2F79005EEE0FF90644AEFF022EC4D6011ED60010C8B938A838982E4F0A3DDFCDCFA75930022EF54016004D2AF8002C2AFEF5402FF9044F4E0545D
:40374000FD4FF0229043A2E0FFEF4404FFEFF09043B2E0FFEF4404FFEFF0229005DCEFF09005DCE0FFEFC43354E0FF904482EFF0229005DCEFF09005DCE0FFEFC43354E01D
:40378000FF904481EFF0229044F4E0F84402F0E85402FF10AF012274014FFF22900642E0FFEF700912362A9006427401F012330222900645E0FFEF700912300B90064574E5
:4037C00001F012397B22900646E0FFEF7009122E0B9006467401F012398722900649E0FFEF7009122E769006497401F012399F2290FFFF120685EFF09046EA7401F0900062
:403800000112068522123A257E307FB81235B67F0712375B123A1E22123A3A7E357F241235D47F07123771123A33229005DBEFF09005DBE0FF9005DBEFF080FE22906569FC
:40384000E0FF9005DCEFF09005DCE0FF22906469E0FF9005DCEFF09005DCE0FF2290645AE0FF9005EEEFF09005EEE0FF229005DEEFF09005DEE0FF906408EFF0229005DE82
:40388000EFF09005DEE0FF906448EFF0229005DEEFF09005DEE0FF906428EFF0229005DEEFF09005DEE0FF906488EFF022906468E0FF9005DEEFF09005DEE0FF229005DF43
:4038C000EFF09005DFE0FF906486EFF022906466E0FF9005DFEFF09005DFE0FF229005DDEFF09005DDE0FF906476EFF0229005DEEFF09005DEE0FF906487EFF02290646792
:40390000E0FF9005DEEFF09005DEE0FF229005DCEFF09005DCE0FF906576EFF0228B938A838982E0FFA3E0FE759300228B938A838982EDF0A3ECF0759300227F0112346D27
:403940007F0A7E001234A0221238ADEF30E405123A6080F4221238CDEF30E4051239D980F4221238FDEF30E4051239E380F4227F0012390D1237DB1238182290647BE0FF3E
:40398000EF4480FFEFF022906575E0FFEF4480FFEFF022906575E0FFEF547FFFEFF022906477E0FFEF4480FFEFF0228B938A838982E0759300FF228B938A838982EDF07589
:4039C000930022EE30E707C3E49FFFE49EFE22122CAA1235F2123805227B027A64795612391F227B027A65795612391F227B027A40798012391F22904082E0FFEF5407FFEA
:403A0000227B027A41790012391F22904102E0FFEF5407FF227F001238DD1237C6229044C07404F0229044C87404F0229044D87404F0229044C07402F0229044C87402F09B
:403A4000229044D87402F02268656C6C6F007F0112343B227F0012343B227F0012346D22906458E0FF22323232325B03432440000049C800150051100010005160001000D1
:403A800051F000100100000A00010A80058001140008000140000A00014C00020001500000200052600809000006010A000809080080000000000000000000000000000005
:403AC00000000000000000000000000000000000000000000000000000000000000000000000000000000000000000000000000000000000000000000000000000000000C6
:403B00000000000000000000000000000000000000000000000000000000000000000000000000000000000000000000000000000000000000000000000000000000000085
:403B40000000000000000000000000000000000000000000000000000000000000000000000000000000000000000000000000000000000000000000000000000000000045
:403B80000000000000000000000000000000000000000000000000000000000000000000000000000000000000000000000000000000000000000000000000000000000005
:0200000480007A
:4000000021005206043018A01920281029322C01006404862D872D882D8A0F006503860F8A728B38010303A620B620EA10010501A62001065503010C0413011E0225022E26
:40004000053004320235023601370138203C2A3F104064410249FF4AFF4BFF4DA04F0450185425580459045A045B045C445D445F05604062C06440654066C068C06AC06C73
:40008000C06EC081018D02920497029801AA02B002B404B501B601B702BC20BD80BE40BF10C034C102C5D0C620C710C82AC9FFCAFFCBFFCDAFCE0FCF04D018D280D425D8CA
:4000C00004D904DA04DB04DC33DD34DF05E040E2C0E440E540E6C0E8C0EAC0ECC0EEC001073A054009020B080F0210081601184019201B801D401E501F10200422402690BA
:400100002F10300835103612384039023C023E103F124120421443014520470149024F105120520359055A805D025E44600465106F03710279407F0287808A80A620C080CB
:40014000C28AC482CA40CC82CE89D0A7D220D6DBD824DE18E40201085802011E011F0123012C0232013402350139023A803E144030410245D04712483249FF4AFF4BFF4DAE
:40018000A04F0450185425580459045A045B045C655D665F01604062C06440654066C068C06AC06CC06EC080EE841285088645870288EC89028A028B088C0F8D018E108FDB
:4001C0000890119103922293049402950299089A809C109D089E689F02A0EEA10AA4EAA604A804A90CAB03AC6AAD0AAE84B007B10FB480B678BA80BB02BE10D440D804D9B1
:4002000004DB04DC22DD20DF010109450004011102400302068009020A3A0D80106A1322178018801A421B121D101F442102220225102780284029202A402E0230083250D3
:400240003302374039944408450446044F0156065C085E805F0161206280632065108208900491159298964099249B439D409E029F04A02AA124A2C8AE02B110B301C01F01
:40028000C28FC48FCA8DCC1FCE0ED060D6D0D82EE084E402EA02010A0E8E019F02A301AC01B001B101B302D280D804D904DB04DC66DD60DF01010B370044010103080602D3
:4002C000082009880A80102011101780180419301A101B081E80211022082504278028202A802B082E023002319032083740388039154060411042C0430449264A8250484C
:4003000051286140682269156A8071807302774089028A04C08FC20FC486CA8ECC1FCE0FD007D20CD80801145704180506062209020C200D060E181101142818121A201E61
:40034000062220240128382A042B0434013506363E370139223D023F50400245014605480549FF4A074BFF4C404D204EF04F055008580459045A045C355D055F01604061BD
:40038000A862406320850288029602970599049B01A402A601A705A904AA06AB01B002B102B204B401B501B704BF01C051C102C5EBC7C0C823C9FFCAFFCBFFCEF0CF44D0FD
:4003C0000CD280D804D904DA04DB04DC11DD45DF01E6C0EA40EB02011542004405100A290E20108011101304171819201A0B1D101E201F16216124082680274029202F142F
:4004000032013718386439103A083B403F044120460847404B044D014E104F40508057017401794080048A808D408F0290649140950396089B189D10A481A610A701AF8046
:40044000B110B301C045C227C46ECA64CC61CE4ED034D210DE08E280E640EA05EC10011659080114011B012002240128013402350136013B2C3E104064410149FF4AFF4BFD
:40048000FF4DA04F045018540156045804590B5A045B045C415D535F01604062C06440654066C068C06AC06CC06EC08419850186268B018C198D018E629302944C960197BE
:4004C000019A77A004AB02AC18AE20AF01B078B101B207B446B502BA2ABF01C064C101C5D0C602C701C816C9FFCAFFCBFFCDAFCE0FCF04D018D804D904DA04DC35DD03DFB0
:4005000001E040E2C0E440E540E6C0E8C0EAC0ECC0EEC001173D004405100A280E2010811501171818641A201E081F8022202340271828012B0931023204371038644180B0
:4005400043014580470149214D205008518053085D115E085F4064406D406F017E8081848440954299209D05A102A280A409A620B304C045C226C479CA0CCC23CE0ED0997F
:40058000D224D6F0D880DE80E602E880EA01EC4001185B03080409050806060B080C030D080E0C10051101120A13461524161017911A101C021E0D253729372D122FA1305B
:4005C00010310733C03530360F370839803A803E013F044034410542064402450C460E480549FF4AFF4BFF4C624DA04EF04F41500C580459045A045C525D055F0166406774
:400600000269106A306B106D106E106F12820184108502862787048C0E8D028E108F0490149106922B95019C389D01A501B003B104B501B63CB702B880BF41D409D804D945
:4006400004DB04DC52DD20DF01011948000401020302048409020A020D0A0E020F1819021A021D401E021F0121212301244025802612271829082C082D482E043008310200
:4006800032403602370838843C023D083E103F40408041014504464047144BC04F585680588059045B21630189208A409084938899049B219D409E80A102A302A580A91060
:4006C000B540B602B704C0ADC2F9CA72CCCBCEFAD0E0D230D60FD808E602EC40011A4205020D0F19091B061D0E1F012106250E27012B012D04330837073B803F0456025731
:400700001259045B045C505D505F0180FE8438850486C4890C8A088CC08D1F903091039480971399029AC69C209D0F9F10A038A108A2C2A4CEA513A630A70CA810A91CAB22
:4007400003AC48AD01AE01B23EB31CB401B50FB6C0BA08BB20D418D804D904DB04DC55DD50DF01011B400440051406400D200E290F8814401540160817041D141E122002B9
:400780002180228425082620270429442B442D402E112F20304031803220332036963A483B803E283F405A085E02670A68086A847140722985028D408E208F40904093CAEE
:4007C0009540969499029F04A120A212A409A508C0F0C2F0C4F0CAFFCCFCCE7AD682D830E418EA05EC10014004320433803480CC7001410553209608A780B480D4200142AF
:400800000B022007103E104D1050409608A7A0C030CE20D220D42001430B111086249480951096189B10A220A7A0C440E440E6100144027C08DE010145019C080146034519
:40084000089C08D00101470882018640880896049C08A508AE04E00101480B2510840487809610A7A0A840B110B710C820E650EA800149155E026140660174047B02820118
:4008800089408E01A004A302AA10AB02AF20B510D6C0D880DC80DE20E680EAA0EE10014C0F1220132017087A407D08862096049A01A104A240A508B504C40EDE03EC0201DD
:4008C0004D1301020A0452026201670887048D028E0296049A01AB28B508C008C202D401D803E202E408EC08015006007C0A180C64103E1A3A1C24015103003F03C0122022
:40090000040100000C00000004840000278400000180060408601300040400802001000031560E090484000000000000040A001000040400000700380000077F38800000FB
:4009400000082800000000103604200005DEFB0C1FFFFFFF2200F008040000000000022004040404222200010000C00040011011C0010011400140010000000000000000CC
:4009800000000000000000003000003505000002020000000C0001C0CD000D0000000000007F7F00000000000000000000E0E0000002020000000000020041323200320087
:4009C00000000000270018010000000000000000000000000000000000000000000000000000000000000000000000000000000000000000000000000000000000000000B7
:400A000000000000000000000000000000000000000000000000000000000000000000000000000000000000000000000000000000000000000000000000000000000000B6
:400A40000000000000000000000000000000000000000000000000000000000000000000000000000000000000000000000000000000000000000000000000000000000076
:400A80000000000000000000000000000000000000000000000000000000000000000000000000000000000000000000000000000000000000000000000000000000000036
:400AC00000000000000000000000000000000000000000000000000000000000000000000000000000000000000000000000000000000000000000000000000000000000F6
:0200000490006A
:0400000000004005B7
:0200000490105A
:04000000BC90ACAF55
:0200000490303A
:02000000936CFF
:0200000490501A
:0C00000000011E02806903011E2313D5BD
:0200000490402A
:4000000000000000000000000000000000000000000000000000000000000000000000000000000000000000000000000000000000000000000000000000000000000000C0
:00000001FF
